:100000000A2883120313B0008A01300801398207DD
:100010000A3400340630831603139F000230850033
:1000200086010030A02183120313AB002B08860049
:10003000AC0183120313AC1B212808302C020318D7
:100040002F282330831203132C07840083130130DD
:100050002B05303E80000310AB0CAC0A19286D2133
:1000600083120313A0002008533A031DDC280A3032
:10007000B000B1012C216D2183120313A1000A30BD
:10008000B000B1012C216D2183120313A2002208BC
:10009000303A03194F28013A03195328572883127D
:1000A00003132D105728831203132D14572883127E
:1000B00003132108413A03197328033A03197E28D0
:1000C000013A03198928073A03199428013A0319B8
:1000D0009F28033A0319AA28013A0319B5280F3AB1
:1000E0000319C028CB28831203132D1C06102D18CA
:1000F000061430302D183130A300CB28831203139F
:100100002D1C86102D18861430302D183130A40087
:10011000CB28831203132D1C06112D180615303021
:100120002D183130A500CB28831203132D1C861106
:100130002D18861530302D183130A600CB288312AB
:1001400003132D1C06122D18061630302D183130D1
:10015000A700CB28831203132D1C86122D18861698
:1001600030302D183130A800CB28831203132D1CFA
:1001700006132D18061730302D183130A900CB2862
:10018000831203132D1C86132D18861730302D185B
:100190003130AA00CB280030A021831203130606B9
:1001A0000319D528AE01060882210A3083120313F1
:1001B000B000B1012C212929831203132008473AEA
:1001C000031D2929F430B0000130B1002C21831225
:1001D0000313AC0183120313AC1BF22808302C026A
:1001E000031823294130831203132C075821503060
:1001F00083120313B000B1012C2183120313AE014B
:10020000B621503083120313B000B1012C212330EA
:10021000831203132C0784008313000858215030E5
:1002200083120313B000B1012C2183120313AE011A
:10023000B621503083120313B000B1012C21831278
:100240000313AC0AEA283930582183120313AE0194
:10025000B6212F2863000A288312031330083104C3
:1002600003194529023083168100833083128100EF
:1002700083120313010803193E293829831203133B
:10028000B003300A0319B1032C2908001F30831270
:100290000313B3003308B200B20B4C2908000F302F
:1002A00083120313B1003108B000B00B55290800C8
:1002B00083120313B0000830B100B00905144621C1
:1002C000B00C031C65290514662905104621B10BE5
:1002D00060290510462100000800851C6D294F216A
:1002E000851C6D290830AF00AE014621AE0CAE175B
:1002F000851CAE13AF0B75294621AE09831203137B
:100300002E08080083120313AF002E0803178D0078
:1003100003132F0803178C0083168C130C158B13F3
:1003200055308D00AA308D008C140A3083120313CF
:10033000B000B1012C218B17831603170C11080094
:1003400083120313AE002E0803178D0083168C133F
:100350000C140A3083120313B000B1012C21831254
:1003600003170C080313AF002F08080083120313B0
:100370002E08012083120313AF0083120313AF086A
:100380000319D329AE0AAF08031DC729D329831245
:1003900003132F085821831203132E080120831200
:0803A0000313AF00BD290800A2
:02400E00022F7F
:00000001FF
